:10000000831606309F00F8308500860183124A204F
:100010006F200E3061209020A60126082720003E88
:100020000319162868209020A60A0D28A60AC030B9
:100030006120902026082720003E031923286820ED
:100040009020A60A1A280130612090200C288207EF
:1000500053345034453443345434523455344D348D
:10006000CE34B034D134CD34DF34B034BC34DE34AB
:10007000003430343134323433343434353436347B
:1000800037343834393441344234433444344534D9
:100090004634003488208820303061208820303079
:1000A00061208120303061208120383061206F2034
:1000B000083061206F20013061206F200630612000
:1000C00008008600851005110514000005100800C1
:1000D000860085100515051400000510080083161C
:1000E000FF308600831205118514051406080510DB
:1000F000A500A51B6F28851083160030860083128B
:100100000800A530A00000000000A00B8528080012
:100110006330A100000000008120A10B8C280800A2
:100120006330A2006230A3000330A40000008820E6
:10013000A20B97288120A30B9A28A40B9D280800C6
:00000001FF
